:100000000C9446000C9466000C9466000C946600F8
:100010000C9466000C9466000C9466000C946600C8
:100020000C9466000C9466000C9466000C946600B8
:100030000C9466000C9466000C9466000C946600A8
:100040000C9466000C9466000C9466000C94660098
:100050000C9466000C9466000C9466000C94660088
:100060000C9466000C9466000C9466000C94660078
:100070000C9466000C9466000C9466000C94660068
:100080000C9466000C9466000C94660085B780683A
:1000900085BF11241FBECFEFD0E1DEBFCDBF11E081
:1000A000A0E0B1E0EAE4F2E100E00BBF02C007909B
:1000B0000D92A030B107D9F711E0A0E0B1E001C086
:1000C0001D92A030B107E1F70C9420060C940000BB
:1000D0002F923F924F925F926F927F928F929F9258
:1000E000AF92BF92CF92DF92EF92FF920F931F9346
:1000F000CF93DF93CDB7DEB726970FB6F894DEBF68
:100100000FBECDBF5C016A017B01522E180127FF93
:1001100002C0552405C085E2821714F485E2582EEA
:10012000D5019896BE83AD8320E030E040E050E0FA
:10013000C701B6010E945E07882354F4F101808153
:100140009181826091838083F7FAF094F7F8F094BC
:10015000AE014F5F5F4FC701B6010E94BE073B0172
:100160004C01E980FA800B811C8120E030E040E006
:1001700050E0C801B7010E945E078823E9F1CD80F5
:10018000DE80442428C02DEC3CEC4CEC5DE3C8013F
:10019000B7010E94EE07AE014F5F5F4F0E94BE079E
:1001A0002AE939E941E251E40E94EE070E9443073F
:1001B000605DD6016E936D014394E980FA800B81F6
:1001C0001C8120E030E040E050E0C801B7010E940F
:1001D0005E07882319F0AC14BD04A8F2750106C0AF
:1001E000F60181916F01D7018D937D01ED81FE8133
:1001F000CE16DF06A8F329C020E030E040E050E052
:10020000C401B3010E94610718161CF07501442453
:100210001CC0442403C04A943701480120E030E068
:1002200040E251E4C401B3010E94EE077B018C015E
:1002300020E030E040E85FE30E945E0787FDEBCFFF
:10024000E982FA820B831C837501D1014D915C9187
:1002500053FF13C0BDEF4B1684F0242D332727FD29
:100260003095852D992787FD909501962817390798
:1002700024F45460F10151834083D1018D919C910C
:1002800092FD08C05394052D112707FD10950A0D06
:100290001B1D0CC0052D112707FD10950A0D1B1DF8
:1002A000842D992787FD9095080F191F0A151B05A6
:1002B000D8F4F5014CC020E030E040E251E4C40144
:1002C000B3010E94EE07AE014F5F5F4F0E94BE0771
:1002D0003B014C0169817A818B819C810E9443079B
:1002E000605DD7016D937D010E151F0528F0ED812E
:1002F000FE81EE16FF06F8F28D819E810817190720
:1003000018F0F50117A224C0D8018C918B5F8C9353
:10031000F80131E318C020E3D8012C93A016B106F0
:1003200028F48E918D018F5F8C930DC0D8013C9382
:100330004394D1018D919C9192FF05C0AE16BF06EA
:1003400008F420833196D8018C918A3324F71082E7
:10035000842D992787FD909526960FB6F894DEBFD9
:100360000FBECDBFDF91CF911F910F91FF90EF9006
:10037000DF90CF90BF90AF909F908F907F906F90C5
:100380005F904F903F902F9008952F923F924F9201
:100390005F926F927F928F929F92AF92BF92CF9215
:1003A000DF92EF92FF920F931F93CF93DF93CDB71E
:1003B000DEB7EE970FB6F894DEBF0FBECDBFCC24EC
:1003C000DD2476013C017EAF6DAF5A011A8219829D
:1003D000FC0117821682838181FDF3C38FEF9FEFAB
:1003E00016C409811A8100FFD3C3842D80538A303B
:1003F000D0F4F0E34F1631F4552021F403FD02C090
:10040000116075C18AE0252D2802C0011124542CE9
:10041000580E30ED530E57FE02C04FE7542E03FD29
:10042000CAC3352CC8C3442D45564CAF433028F0C1
:10043000842D8554833008F0FCC0C501049698AF24
:100440008FABF501C080D180E280F38003FD02C054
:1004500036E0532E077B1A83098346015701A70113
:100460009601C701B6010E9428068823C1F08EE4D8
:100470008D838B8381E48C839E012A5F3F4F3AAF4B
:1004800029AF3CAD333008F07AC28B81805E8B831C
:100490008C81805E8C838D81805E8D8370C2C7016C
:1004A000B6010E94B507892BE9F089E48D838EE4BB
:1004B0008C8386E48B8320E030E040E050E0C7018D
:1004C000B6010E945E0787FD06C0AE014A5F5F4F1E
:1004D0005AAF49AFD6CF8DE28E83CE0107969AAF41
:1004E00089AFCFCFC80192609A838983E7E44E1623
:1004F00009F449C0E41544F0F5E44F1679F026E418
:10050000421609F042C31DC036E64316D1F047E655
:100510004416C9F155E6451609F037C38E010F5F41
:100520001F4F252DB501A401CE010F960E94680032
:10053000282E8CEF380E15140CF43A94DE011F9619
:1005400015C094609A8389838E010F5F1F4F252DFC
:10055000B501A401CE010F960E946800282E151443
:100560000CF43A94DE011F96121444F4FD0101903C
:100570000020E9F73197CE2ECA1A02C0C52CC394C9
:10058000BAAFA9AF7DC1552011F0252D01C021E0E2
:1005900098609A8389838E010F5F1F4FB501A40174
:1005A000CE010F960E946800282E89819A8192FFC1
:1005B0001EC0822D850D8150282FA82FBB27A7FD97
:1005C000B095AC0FBD1F1F9605C08C91119721509F
:1005D000803331F4622F27FD23C02215B4F703C303
:1005E000C62E562E5218539400C3C92E17C0252D5F
:1005F000E52DFF27E7FDF095EC0FFD1F3F9606C0A8
:1006000080813197292F2150803379F7922F12164C
:10061000BCF3522EC22E222309F4EFC2592EEDC292
:10062000E22FFF27E7FDF095EC0FFD1F108A552400
:1006300099CFC8018870907003FF04C0552011F451
:1006400021E0522EE9E64E1609F493C0E4153CF180
:10065000F3E54F1609F474C0F415ACF02BE2421622
:10066000E1F1241544F030E24316D1F143E244169F
:1006700009F080C23FC05DE24516C1F18EE2481626
:1006800009F078C239C093E64916E1F1E4E64E1666
:1006900009F46FC0F8E54F1609F06CC29FC020E75F
:1006A000421609F496C0241544F03CE6431641F185
:1006B0004FE6441609F05EC20DC055E7451609F431
:1006C0008FC0E8E74E1609F489C0F3E74F1609F02A
:1006D00051C221C028E02BAF83C000611A83098377
:1006E00089819A8180629A83898365C200681A83AE
:1006F000098361C20064FBCF08601A83098352C278
:100700000460F5CFA5014E5F5F4F58AF4FABF501C9
:10071000C0803A9434C1F501C080D180892B41F06A
:10072000652D772767FD7095C6010E940B0718C0DD
:10073000F60101900020E9F73197EC19EBAF11C0F9
:10074000F501C080D180892B41F0652D772767FDA9
:100750007095C6010E94000703C0C6010E94F706FB
:100760008BAF95012E5F3F4F38AF2FAB3BAD331AA8
:1007700006C102FF0BC0A5014C5F5F4F58AF4FABE6
:10078000F50160817181828193810EC095012E5F98
:100790003F4F38AF2FABF501808191819C01B901AA
:1007A000882777FD8095982F6B017C0197FF0BC000
:1007B00002601A830983F094E094D094C094C11C21
:1007C000D11CE11CF11C89819A818F7B9A838983DA
:1007D00027C000641A83098398E7492E30E13BAFB4
:1007E00029813A8122FF0BC0A5014C5F5F4F58AFB2
:1007F0004FABF50160817181828193810CC0A501AD
:100800004E5F5F4F58AF4FABF50180819181AC01D6
:10081000BA01882799276B017C012F7C3A832983B1
:1008200087017601CE0103969AAF89AF9BADA92EC1
:10083000BB24CC24DD24C801B701A60195010E9488
:10084000B8086A301CF0640D615201C0605DE9AD0A
:10085000FAAD6193FAAFE9AFC801B701A6019501FE
:100860000E94B80879018A01211531054105510519
:1008700011F7CC24DD247601CE010396C9ACC81A49
:1008800049815A81CA0182739070892B09F03A9488
:1008900046FF07C0FBADF03111F482E001C081E0FA
:1008A000381A43FF10C0252D332727FD30958C2D96
:1008B00099278217930724F0477F5A83498303C0FF
:1008C0005C18351801C03C1840785170452B69F40C
:1008D000832D06C0B30180E290E00E941607812FAD
:1008E000182F11501816B4F3312E89819A8181FF87
:1008F00004C0B3018DE290E00BC084FF04C0B301DB
:100900008BE290E005C085FF05C0B30180E290E076
:100910000E94160789819A8186FF0FC0B30180E388
:1009200090E00E9416072BAD203139F4B301842DDD
:10093000992787FD90950E94160789819A8190FFDB
:100940000DC0832D06C0B30180E390E00E9416071E
:10095000812F182F11501816B4F3312E89819A81E6
:1009600083FF0DC0252D06C0B30180E390E00E94F7
:100970001607212F122F11501216B4F3512E898110
:1009800087FD0DC0832D06C0B30180E290E00E9478
:100990001607812F182F11501816B4F3312E33E695
:1009A000431631F4B3018C2D992787FD9095BEC075
:1009B00043E74416B1F4460156011BAD09C0F501E9
:1009C00081915F01B301992787FD90950E941607D9
:1009D0001150A8F76401FBADCF0ED11C2FEF2BAF48
:1009E000B8C033E54316B1F446018601BBAC08C07C
:1009F000F8018491B30199270E9416070F5F1F4FDA
:100A0000BA94FFEFBF16A1F764012BADC20ED11C43
:100A1000FBAF9FC089819A8191FD03C009AD1AADDA
:100A200091C092FF1DC01214BCF4A9ACBAAC122D37
:100A300009C0F50181915F01B301992787FD909568
:100A40000E9416071150A8F729AD3AAD220D311DAD
:100A50003AAF29AF22240FC0B30180E390E009C070
:100A6000E9ADFAAD8191FAAFE9AFB301992787FDFE
:100A700090950E94160715142CF4B3018EE290E0B5
:100A80000E94160789819A8192FD06C017C0B301A2
:100A900080E390E00E9416072394822D815087FF07
:100AA0000DC05A94852D8F5F18168CF307C0B301C3
:100AB000892F992787FD90950E941607E9ADFAAD19
:100AC0009191FAAFE9AF992329F05A94852D8F5F60
:100AD00018166CF389819A8192FD3BC0B301842D75
:100AE000992787FD90950E9416072A9427FE07C034
:100AF000B3018DE290E00E941607219405C0B30176
:100B00008BE290E00E9416076AE070E0822D992740
:100B100087FD90950E94A5086B017C01CB01C096D2
:100B2000B3010E941607B301C701C0960E941607C1
:100B300010C0F80182918F01B301992787FD90952C
:100B40000E941607CE0103960817190791F71AAFEE
:100B500009AF898187FF17C0832D06C0B30180E2EA
:100B600090E00E941607812F182F11501816B4F329
:100B7000312E09C0B301842D992787FD90950E94DD
:100B80001607B8AEAFAA1A821982AFA8B8AC13C0C4
:100B9000F5E24F1649F481E090E09A8389832AE0D8
:100BA0002BAF3324552407C0B301842D992787FD2B
:100BB00090950E9416074DAD5EAD4F5F5F4F5EAFE3
:100BC0004DAFF301838183FF04C0EDADFEAD4490D2
:100BD00003C0EDADFEAD4080442009F002CCF3012E
:100BE0008681978114C0C22E5524EC2DFF27E7FD86
:100BF000F095EC0FFD1F108AB2CCEC2DFF27E7FD1E
:100C0000F095EC0FFD1F108AFEEF4F0E92CCEE9682
:100C10000FB6F894DEBF0FBECDBFDF91CF911F910D
:100C20000F91FF90EF90DF90CF90BF90AF909F908B
:100C30008F907F906F905F904F903F902F9008958E
:100C4000CFEFD0E1DEBFCDBF8AEB809300F0FFCFC6
:100C5000A8E1B0E0EEE2F6E00C94FE0869837A8346
:100C60008B839C832D833E834F835887BE01675FB0
:100C70007F4FCE0101960E945806BE016F5E7F4FE6
:100C8000CE0105960E9458068985823018F481E0CD
:100C900090E00AC020E030E08989823010F0C9017C
:100CA00003C021E030E0C901E2E068960C941A0923
:100CB000FC01DB01208131819281492F4F7750E087
:100CC000991F9927991F8381682F660F692B881FA9
:100CD0008827881FFD018183662309F049C02115FB
:100CE00031054105510509F470C082E89FEFFD010F
:100CF00093838283220F331F441F551F220F331FFC
:100D0000441F551F220F331F441F551F220F331F2F
:100D1000441F551F220F331F441F551F220F331F1F
:100D2000441F551F220F331F441F551F83E08C9310
:100D30002030F0E03F07F0E04F07F0E45F0790F469
:100D400082E89FEF220F331F441F551F0197203069
:100D500060E0360760E0460760E4560798F3FD015F
:100D600093838283FD0124833583468357830895CB
:100D70006F3F71F1862F99278F579040FD01938324
:100D8000828383E08C93220F331F441F551F220F51
:100D9000331F441F551F220F331F441F551F220F9F
:100DA000331F441F551F220F331F441F551F220F8F
:100DB000331F441F551F220F331F441F551F5064FC
:100DC0002483358346835783089582E08C93089566
:100DD000211531054105510519F484E08C930895DE
:100DE00044FD02C01C92BECF81E08C93BBCFFC01BE
:100DF00005900020E9F7809590958E0F9F1F08952C
:100E0000FC010590615070400110D8F780959095D5
:100E10008E0F9F1F0895FC016150704001900110DA
:100E2000D8F7809590958E0F9F1F08950F931F936D
:100E3000CF93DF938C01EB018B81992781FF1BC03E
:100E400082FF0DC02E813F818C819D81281739073B
:100E500064F4E881F9810193F983E88306C0E885A9
:100E6000F985802F0995892B31F48E819F81019618
:100E70009F838E8302C00FEF1FEFC801DF91CF91D8
:100E80001F910F91089597FB47D09F3738F0FEE9E7
:100E9000F91B982F872F762F6B2F05C05AC0969578
:100EA000879577956795F150D0F73EF490958095AA
:100EB000709561957F4F8F4F9F4F08950ED05EF0D4
:100EC00004C00BD026F001C008D019F020F48FEF39
:100ED000089580E0089581E0089597FB092E052686
:100EE00000F8689410D0E89407FC07C062177307F5
:100EF0008407950721F008F40094079498940895C6
:100F0000052E092607FA440F551F5F3F79F0AA27DF
:100F1000A51708F051E04795880F991F9F3F31F0C2
:100F2000BB27B91708F091E0879508959F919F918D
:100F3000112408C197FB880F991F9F3F31F0BB27F1
:100F4000B91708F091E0879508959F919F9111241A
:100F5000F9C0662777278827992708959F3F59F476
:100F6000803C49F481E0992708959068892387237C
:100F700086238395B9F3882799270895DBDFCF93DC
:100F8000DF93D52FC42F55274427332722279923B2
:100F9000D9F09F37C8F0F92FBDD0592F482F372FE0
:100FA000262FF63968F46FDFA6D0C030CD0721F0C8
:100FB00069937993899399939058DF91CF9157C012
:100FC0009927882777276627C030CD0721F02993F6
:100FD000399349935993DF91CF919CC091DF01D010
:100FE00099C0992339F0552329F09F575F57950FE2
:100FF00013F49AF1B1CF91589F3FE1F3629FA12D75
:101000000F92BB27639FA00DB11DEE27729FA00D0D
:10101000B11DEE1FAF93AA27649FB00DE11D739F12
:10102000B00DE11DAA1F6627829FB00DE11DA61F0E
:101030005527749FE00DA11D551F839FE00DA11D35
:10104000561F849FA00D511D852F7A2F6E2F1F9044
:101050000F9088231AF4939539F474C0000C111C76
:10106000BB1F661F771F881F012808955058192E2F
:1010700047DF01D04FC0BA1762077307840795078F
:10108000B1F188F40EF410940B2EBA2FA02D062E79
:10109000622F202D072E732F302D082E842F402DE8
:1010A000092E952F502DFF275523B9F0591B49F0D4
:1010B000573E98F0469537952795A795F04053955C
:1010C000C9F776F0BA0F621F731F841F30F487953B
:1010D00077956795B795F040939517FA0F2E089579
:1010E000BF1BBB27BA0B620B730B840BF6CFDEF66C
:1010F00033CFE89403C097FB0EF4D8DEB62F672FEA
:10110000782F892F9EE9002405C09A95BB0F661F92
:10111000771F881F11249923A1F08823B2F79F3FDE
:1011200059F0BB0F48F421F4002011F460FF04C013
:101130006F5F7F4F8F4F9F4F881F9795879597F9C8
:10114000089507CF9FEF80EC089597FB092E07269F
:101150000AD077FD04D02ED006D000201AF4709566
:1011600061957F4F0895F6F7909581959F4F08956B
:10117000A1E21A2EAA1BBB1BFD010DC0AA1FBB1F9B
:10118000EE1FFF1FA217B307E407F50720F0A21B0D
:10119000B30BE40BF50B661F771F881F991F1A947A
:1011A00069F760957095809590959B01AC01BD01A4
:1011B000CF010895AA1BBB1B51E107C0AA1FBB1F8B
:1011C000A617B70710F0A61BB70B881F991F5A95D3
:1011D000A9F780959095BC01CD0108952F923F927B
:1011E0004F925F926F927F928F929F92AF92BF9237
:1011F000CF92DF92EF92FF920F931F93CF93DF93E3
:10120000CDB7DEB7CA1BDB0B0FB6F894DEBF0FBE3F
:10121000CDBF09942A88398848885F846E847D848C
:101220008C849B84AA84B984C884DF80EE80FD808E
:101230000C811B81AA81B981CE0FD11D0FB6F89404
:0A124000DEBF0FBECDBFED01089523
:00000001FF
